:100000000C94B2020C94CF020C94CF020C94CF0249
:100010000C94CF020C94CF020C94CF020C94CF021C
:100020000C94CF020C94CF020C9463220C943523D1
:100030000C94301D0C94CF020C94CF020C94CF0280
:100040000C94CF020C94CF020C94CF020C94CF02EC
:100050000C94CF020C94B81D0C94CF020C94CF02D8
:100060000C94CF020C94CF020C94CF020C94CF02CC
:100070000C94CF020C94CF020C94CF020C94CF02BC
:100080000C94CF020C94CF020C94CF020C94CF02AC
:100090000C94CF020C94CF020C94CF020C94CF029C
:1000A0000C94CF020C94CF020C94CF022B032E039E
:1000B0003103340337033A033D033405390543055F
:1000C00037053C0541053F051E091E094A094A0935
:1000D000AB09C909E00AE00AD4096D0A7E0A7E0A62
:1000E000A223C923C124C923C12415243824C1242F
:1000F0008F249E246572676F646F785F657A2F64C2
:10010000656661756C74204020302E31352E323199
:100110002D33382D67646136383038002E004C009E
:100120002A00E100354100001E00140004001D619A
:1001300034004D001F001A0016001B00E1042A00C5
:10014000200008000700060050002C0021001500C8
:10015000090019004F004A00220017000A0005009C
:1001600000006564500001530000006F0000E300D0
:100170004F000153000000670000E20023001C0054
:100180000B00110000002961240018000D00100070
:1001900052004B0025000C000E00360051002800D4
:1001A000260012000F0037002F002B00270013003D
:1001B0003342386130004E002D0031003468E500D4
:1001C00001580000A75D010001000100DF5C000094
:1001D0003A001E0220022202010001003B001F0221
:1001E000210223020100CA5C3C002F0226022F00DC
:1001F0000100CB5C3D00300227023000010001000D
:100200003E003102350035020000C45C01000100EF
:1002100000000100000001000100010000000100D9
:100220000000C35C3F005200510024020000CE5C7D
:100230004000240021001E000100010041002500B3
:1002400022001F003700C65C420026002300200069
:100250002700C75C430025022E0231002E0001005A
:100260004400450001000100010000000100010000
:100270000100010001000000010001000100010077
:100280000100010001000100EF0001000100010078
:100290000100ED00EE000100F1000100010001008D
:1002A000F0000100F2000100010001000100010066
:1002B0000000010001000100000001000000010039
:1002C0000100010000000100000001000100010028
:1002D0000100010000000100010001000100010017
:1002E000A9000100010001000100AC00AA00B60055
:1002F000010001000100AB00A800010001000100A5
:10030000010001000100010001000100AE00010038
:100310000100000000000000000000002A2B28005F
:1003200000000000000000000000000000000029A4
:10033000000000002C1E3420212224342627252EE4
:10034000362D3738271E1F2021222324252633331C
:10035000362E37381F0405060708090A0B0C0D0E48
:100360000F101112131415161718191A1B1C1D2F14
:100370003130232D350405060708090A0B0C0D0E34
:100380000F101112131415161718191A1B1C1D2FF4
:100390003130354C0000000000000000000000007B
:1003A000000000000000000000000000000000004D
:1003B00000000000000000007E0F00D4FFFFFFC718
:1003C0000000007816034500720067006F004400CB
:1003D0006F007800200045005A00000028035A00F2
:1003E00053004100200054006500630068006E0067
:1003F0006F006C006F006700790020004C00610006
:1004000062007300000004030904090254000301A0
:1004100000A0FA09040000010301010009211101F3
:1004200000012240000705810308000109040100C2
:100430000103010200092111010001224700070503
:1004400082030800010904020001030000000921E1
:1004500011010001226D0007058303200001120134
:1004600000020000000897327449010001020001F7
:1004700005010980A101850319012AB7001501268C
:10048000B700950175108100C0050C0901A1018517
:100490000419012AA002150126A0029501751081F8
:1004A00000C005010906A1018506050719E029E735
:1004B000150025019508750181020507190029EF2E
:1004C0001500250195F0750181020508190129051E
:1004D000950575019102950175039101C00501090A
:1004E00002A1010901A1000509190129081500252A
:1004F0000195087501810205010930093115812531
:100500007F95027508810609381581257F9501754B
:10051000088106050C0A38021581257F95017508AA
:100520008106C0C005010906A101050719E029E7F8
:100530001500250195087501810295017508810155
:100540000507190029FF150026FF0095067508818B
:100550000005081901290595057501910295017598
:10056000039101C011241FBECFEFDAE0DEBFCDBF83
:1005700011E0A0E0B1E0E6E3FDE402C005900D92D9
:10058000A239B107D9F722E0A2E9B1E001C01D927A
:10059000A53EB207E1F70E9420160C9499260C9410
:1005A00000008098889A8198899A84988C9A859876
:1005B0008D9A86988E9A87988F9A08952098289871
:1005C0002198299822982A9823982B9852985A98DB
:1005D00053985B983E9846980895CF93E82F8730BC
:1005E00080F58091060190910701892B09F047C0A1
:1005F000CE2F64E670E080E40E94F91A9093070120
:1006000080930601892BD1F464E670E082E10E94B8
:100610007A1B9093070180930601892B79F481E07E
:1006200090E001C0880FCA95EAF764E670E0809513
:100630000E947A1B9093070180930601CF910C943E
:10064000CF1B90E0FC013797E730F105C0F4EA5A80
:10065000FF4F0C941D25209A289811C0219A2998A3
:100660000EC0229A2A980BC0239A2B9808C0529A3F
:100670005A9805C0539A5B9802C03E9A4698CF910B
:100680000895CF93873040F580910601909107013E
:10069000892B59F564E670E081E40E94F91A909381
:1006A000070180930601892B11F0C0E011C084E698
:1006B00090E00E94AA1B97FF05C0909307018093CA
:1006C0000601F3CFC82FC0951092070110920601C2
:1006D0000E94CF1B8C2F0AC09FB18FB1807F86955F
:1006E00086959370892B809501C080E0CF91089505
:1006F0000E94780490E090930701809306010E9485
:10070000DE020C94D102EF92FF920F931F93CF93CE
:10071000DF938091060190910701892B91F08091E0
:1007200094018F5F8093940181110BC00E94780423
:1007300090E09093070180930601892B11F40E94A9
:10074000EA0304EB12E0C0E0F12C87E0E82EEC0EA7
:100750008C2F0E94ED028E2D0E94ED028C2F0E94A4
:1007600041038F73F8019081891719F08083D1E0DC
:1007700001C0D0E08E2D0E9441038F73F801978154
:10078000891719F0878381E001C080E0D82BFD2A0A
:100790000E94DE02CF5F0F5F1F4FC730B1F68F2D73
:1007A000DF91CF911F910F91FF90EF9008950E94DC
:1007B000780490E090930701809306010E94DE0286
:1007C0000E94D102E2ECF2E0119282E0E03DF807F3
:1007D000D9F7089556985E9825982D9826982E98C2
:1007E00027982F988FEF90E090938900809388004E
:1007F00090938B0080938A0090938D0080938C005F
:10080000259A2D9A2FEF80E792E02150804090406A
:10081000E1F700C00000269A2E9A2FEF80E792E0C1
:10082000215080409040E1F700C00000279A2F9AA5
:100830002FEF80E792E0215080409040E1F700C028
:10084000000025982D982FEF80E792E021508040FE
:100850009040E1F700C0000026982E982FEF80E727
:1008600092E0215080409040E1F700C000002798BE
:100870002F9856985E9825982D9826982E98279808
:100880002F98089589EA8093800089E08093810001
:1008900024982C983F988AB18F7C8AB96E98479A91
:1008A0008BB180638BB9769A0E94D9116093AE02A6
:1008B0007093AF028093B0029093B10267708FEF94
:1008C000689FB00111247595679575956795772791
:1008D000709389006093880070938B0060938A0006
:1008E00070938D0060938C000E94EA030C94551560
:1008F00080E290E09093070180930601809195013A
:1009000081110EC00E94F31A81E0809395012FEFB0
:1009100083ED90E3215080409040E1F700C000005B
:1009200064E670E080E40E94F91A909307018093D6
:100930000601892B09F04EC064E670E080E00E9459
:100940007A1B9093070180930601892B09F042C01E
:1009500064E670E080E00E947A1B90930701809328
:100960000601892BB9F564E670E08FE30E947A1BDB
:100970009093070180930601892B61F50E94CF1B9C
:1009800064E670E080E40E94F91A90930701809376
:100990000601892BF9F464E670E08CE00E947A1B72
:1009A0009093070180930601892BA1F464E670E01F
:1009B00080E00E947A1B9093070180930601892BA7
:1009C00049F464E670E08FE30E947A1B909307017C
:1009D000809306010E94CF1B80910601089510921A
:1009E000AE021092AF021092B0021092B10284E0F7
:1009F00080618093AE026091AE027091AF028091EF
:100A0000B0029091B1020E94DD110C94E9110C9496
:100A100053159C01FB018281882349F0273A3D450B
:100A200039F484EF90E00E94DD0680E0089581E0D3
:100A300008950895CF92DF92EF92FF926B017C01AF
:100A400056985E9825982D9826982E9827982F9836
:100A50000E94E00690E0FC013197E730F105A8F430
:100A6000E35AFF4F0C941D25259A2D9A0EC0259A06
:100A70002D9A269A2E9A09C0259A2D9A04C0259A55
:100A80002D9A269A2E9A279A2F9AC701B601FF907F
:100A9000EF90DF90CF90089581E008950C940905C0
:100AA00008950C9450051F93CF93DF9300D000D08E
:100AB0001F92CDB7DEB749835A836B83309197017C
:100AC00089819A81311114C0662359F0222349F09B
:100AD0000E941F0D182F682F89819A810E94C60CD1
:100AE00003C00E94F20C182F69817A81812F04C003
:100AF0000E941F0D69817A810F900F900F900F90C7
:100B00000F90DF91CF911F910C943514FC01262F8B
:100B1000408151816281738184810C94530581E00D
:100B20000895CF93DF93EC0160E00E948605BE013B
:100B3000DF91CF910C9451050C9442040C9407055D
:100B400008950E94700B0E94A0052FEF84E39CE0A3
:100B5000215080409040E1F700C000000C94DE1D61
:100B60000F931F93CF93DF938C0161E00E94860562
:100B7000EC01B8010E944E058823F1F1B801CE01C5
:100B80000E94A11A8823C1F1B801CE010E94B518B4
:100B9000882391F1B801CE010E94FD19882361F1EB
:100BA000F8018281882309F1CB358DE5D807C1F0A2
:100BB00050F4C115FCE5DF0781F0CF3DDC45A9F419
:100BC0000E944D1219C0CC35EDE5DE0761F0CD3540
:100BD000DD4559F40E94991108C00E94A1050CC07E
:100BE0000E94A21102C00E94A511C801DF91CF91FD
:100BF0001F910F910C944C0580E0DF91CF911F91D4
:100C00000F9108950E94151D0C9441070E944407FE
:100C10000C94191DDF92EF92FF920F931F93CF93C5
:100C2000DF93E82FF0E0EC5EFC4FD490282F269560
:100C30002695269530E0F901EC54FC4F049187701D
:100C400010E0082E02C0159507950A94E2F701708E
:100C50001127F901EC55FC4FE490F12C082E02C04D
:100C6000F594E7940A94E2F791E0E922FF24F90170
:100C7000EC56FC4FC491D0E002C0D595C7958A953B
:100C8000E2F7C170DD270115110519F081EE0E9410
:100C9000A307E114F10419F086EE0E94A3078D2D3D
:100CA0000E94CC08EF2819F086EE0E944D08012B17
:100CB00019F081EE0E944D08CD2B51F08CE2DF91AE
:100CC000CF911F910F91FF90EF90DF900C94CC0883
:100CD000DF91CF911F910F91FF90EF90DF900895DA
:100CE000EF92FF920F931F93CF93DF938C01F62E19
:100CF0008AE0E82EF8018491882309F457C08130F6
:100D000009F042C0E8012196FE018491813031F45E
:100D10002196FE0184910E94CC0839C0823039F4BA
:100D2000E8012296FE0184910E94A30730C083301F
:100D300039F4E8012296FE0184910E944D0827C0F3
:100D4000843029F5E8012296FE01249180E090E0AC
:100D500030E0205331092A30310560F4E89EA001CB
:100D6000E99E500D1124C901840F951F2196FE01A3
:100D70002491EECF009759F0EFE9FFE03197F1F7BA
:100D800000C000000197F6CF0E940A06E8018E011C
:100D90000F5F1F4F8F2D882309F4ACCFEFE9FFE0E1
:100DA0003197F1F700C000008150F5CFDF91CF916E
:100DB0001F910F91FF90EF90089560E00C947006E2
:100DC000CF92DF92EF92FF926C01EE24FF24C114C8
:100DD000D104E104F10421F0C701B60120E101C012
:100DE00020E0C72ED82EE92EFF24C114D104E1043F
:100DF000F10419F0285FC701B6016B017C0154E0D2
:100E0000F694E794D794C7945A95D1F7C114D104B6
:100E1000E104F10419F02C5FC701B6016B017C01FC
:100E200042E0F694E794D794C7944A95D1F7C11459
:100E3000D104E104F10419F02E5FC701B601DC0111
:100E4000CB01B695A79597958795892B8A2B8B2BE8
:100E500009F02F5F822FFF90EF90DF90CF900895E1
:100E600008950C94300781E008950C943307089599
:100E7000CF93C82F0E9431078C2F0E943507CF9146
:100E8000089580E00C9438070E94DD1B0C9438070D
:100E90000E94DD1B90919601891721F080939601A5
:100EA0000C9438070895CF93DF93CDB7DEB72B9717
:100EB0000FB6F894DEBF0FBECDBF4F83588769874A
:100EC0007A878B8761110E94E5109E012F5F3F4F4B
:100ED00086E0F90111928A95E9F785E0FE013796DF
:100EE000D90101900D928A95E1F789819A814C810F
:100EF0005D81452B31F09F3F31F491E08F3F19F434
:100F000003C091E001C090E090FF09C049815A817F
:100F10006B817C818D819E810E94061005C0C90174
:100F20000E948F058111F2CF2B960FB6F894DEBF89
:100F30000FBECDBFDF91CF910895FC0180819181DB
:100F40000E94610D0895CF93882309F4A4C0C82F8F
:100F50008238C1F40E94DD1B81FD9DC069E3809150
:100F60000A0190910B010E94D01C0E9407112FEFE3
:100F700081EE94E0215080409040E1F700C00000F5
:100F800069E319C0833801F50E94DD1B80FD83C031
:100F900063E580910A0190910B010E94D01C0E9490
:100FA00007112FEF81EE94E0215080409040E1F74F
:100FB00000C0000063E580910A0190910B010E943E
:100FC000DB1CCF910C9407118438C1F40E94DD1B07
:100FD00082FD61C067E480910A0190910B010E943B
:100FE000D01C0E9407112FEF81EE94E02150804029
:100FF0009040E1F700C0000067E4DDCF8CEF8C0F7C
:10100000813AD0F46C2F80910A0190910B010E94DB
:10101000501C882349F06C2F80910A0190910B019C
:101020000E94DB1C0E9407116C2F80910A01909195
:101030000B010E94D01CC5CF80E28C0F883048F491
:10104000C77081E001C0880FCA95EAF70E94C810F6
:10105000B8CFEBE5EC0FE33040F4F0E0E25BFE4F9D
:10106000808190E0CF910C940E1CE8E5EC0FE73105
:1010700050F4F0E0EE0FFF1FE05EFE4F80819181A3
:10108000CF910C94241CCD3E30F08C2F0E94A516DD
:10109000CF910C947717CF910895882309F464C0F9
:1010A000823879F40E94DD1B81FF5EC069E3809184
:1010B0000A0190910B010E94D01C0E94071169E364
:1010C00010C08338B1F40E94DD1B80FF4DC063E582
:1010D00080910A0190910B010E94D01C0E9407117F
:1010E00063E580910A0190910B010E94DB1C0C9436
:1010F0000711843879F40E94DD1B82FF35C067E454
:1011000080910A0190910B010E94D01C0E9407114E
:1011100067E4E7CF9CEF980F913A10F4682FE1CF86
:1011200090E2980F983050F4877091E001C0990FC9
:101130008A95EAF7892F0E94CE10D9CF9BE5980FA8
:10114000933020F480E090E00C940E1C98E5980F0A
:10115000973120F480E090E00C94241C8D3E20F028
:101160000E9400170C94771708951F93CF93DF9375
:10117000182FEB010E94A307209741F08FE99FE011
:101180000197F1F700C000002197F6CF812FDF9182
:10119000CF911F910C944D08893319F060E070E0F5
:1011A00002C060E570E00C94B508882321F00E942D
:1011B000C8100C9407110895882321F00E94CE10C6
:1011C0000C9407110895CF92DF92EF92FF920F9344
:1011D0001F93CF93DF937C01D62FC72FFC01128181
:1011E000058102950F700E94BE108823B9F011236B
:1011F000A9F08C2F807F803421F080E28D0F883021
:1012000068F08091B30282FD09C082E00E946711FC
:101210000E94BE1091E0D82ED92601C0D12CCC2E30
:10122000C2948FE0C8228C2D90E08C30910508F09C
:10123000C7C1FC01EC59FF4F0C941D258C2F807FFA
:10124000CF70882311F0C295C07F112399F0CC2371
:1012500009F4A2C180E28D0F883010F0D11104C0D2
:101260008C2F0E94C81003C08C2F0E94D8100E949F
:10127000071192C18D2F0E944D08CC2309F4A0C103
:1012800080E28D0F883038F1DD2329F18C2F0E9408
:10129000DE1024C08C2F807FCF70803211F0C29579
:1012A000C07FDD2319F0D130A1F13FC08091B3029E
:1012B00082FF17C0112349F0CC2329F08C2F0E9404
:1012C000C8100E94071180E068C180E00E944D08AC
:1012D000CC2309F475C18C2F0E94CE100E940711F7
:1012E0006FC1112371F0002341F0013031F40E94ED
:1012F000E8108C2B0E94F01063C10E94E8108C2B28
:101300000EC0002319F0013009F45AC10E94FD10EB
:101310001EC0112339F0023008F052C18C2F0E94F8
:10132000D5084EC101114CC112C0112319F0002380
:10133000A9F332C1002359F0D93309F03EC1FFEFC0
:1013400007EE13E0F15000401040E1F734C18C2F5C
:101350000E94DC0835C18C2F86958695837019F024
:10136000813061F02DC1112321F08D2F9C2F9370BE
:1013700002C080E090E00E940E1C2AC1112321F0DF
:101380008D2F9C2F937002C080E090E00E94241C5F
:101390001FC18D2F112319F00E94A51602C00E94B3
:1013A00000170E94771714C18C2F837009F047C073
:1013B00011110AC12D2F229526952770220F220F79
:1013C0006D2F6F70862F90E0A0E0B0E0022E04C079
:1013D000880F991FAA1FBB1F0A94D2F7D4FF10C011
:1013E0004FE050E060E070E004C0440F551F661FFE
:1013F000771F2A95D2F7409550956095709503C058
:1014000040E050E0BA01C695C695C3708A019B01C1
:10141000082B192B2A2B3B2BC901B801C23049F0EC
:1014200058F4C13019F00E94DC0BCEC00E94CA0BE8
:10143000CBC00E94EE0BC8C00E94C80BC5C01123D0
:1014400019F08C2F817001C08695882309F4BCC0E7
:101450002D2F229526952770220F220F6D2F6F704A
:10146000862F90E0A0E0B0E0022E04C0880F991F04
:10147000AA1FBB1F0A94D2F7D4FF10C04FE050E060
:1014800060E070E004C0440F551F661F771F2A9567
:10149000D2F7409550956095709503C040E050E0BC
:1014A000BA01C695C695C3708A019B01082B192BFA
:1014B0002A2B3B2BC901B801C23049F058F4C13086
:1014C00019F00E94A10C80C00E948F0C7DC00E9468
:1014D000B30C7AC00E94020C77C0CF70112339F090
:1014E0008C2F0E94280C8D2F0E94D5086DC08D2F47
:1014F0000E94DC088C2F0E94490C66C0D23F19F173
:1015000028F4D03F41F0D13FB9F042C0D33F11F1B0
:10151000D43F71F03DC0112339F0011151C08C2F1F
:101520008F710E946E0C4CC0023008F049C0F7CF9A
:101530008091B30282FF18C0112339F08C2F8F7174
:101540000E94280C3DC01123C9F38C2F8F710E947B
:10155000490C36C0112329F08C2F8F710E94130C77
:101560002FC00E940E0C2CC0112349F0CF718C2F7C
:101570000E94280C63E08C2F0E944C1121C081E056
:101580000E9467110230E0F082E00E94671118C0EB
:10159000112331F0002391F28D2F0E94A30710C078
:1015A000002399F2D93349F41FEF27EE33E01150AD
:1015B00020403040E1F700C000008D2F0E944D0810
:1015C00088EF8C0D843020F40E94DD1B0E943807C8
:1015D000DD20C9F00E94BA1080FD15C0F70112820B
:1015E0000E94B4100E94280CC7010E94240B0E9484
:1015F000B410DF91CF911F910F91FF90EF90DF908A
:10160000CF900C94490CDF91CF911F910F91FF90D7
:10161000EF90DF90CF9008950F931F93CF93DF93B8
:10162000EC01688179818A810E946C0D8C010E9495
:10163000C50C0E94B60BB801CE010E94E308DF91F1
:10164000CF911F910F910895CF93DF93EC01988173
:1016500089812B813C81232B31F08F3F31F481E054
:101660009F3F19F403C081E001C080E080FD1DC0F0
:10167000CE010E94B005811110C00E94BE108823C7
:10168000A1F08A81882389F08091B30282FD0DC088
:1016900082E0DF91CF910C946711CE010E940C0B78
:1016A000CE01DF91CF910C949105DF91CF910895F8
:1016B00080E090E00E940E1C80E090E00E94241CDC
:1016C0000E94E5100E9407110E94A7180C9477173A
:1016D00080910A0190910B010E94E61C0C94580B1A
:1016E0000E94D5100C94680B92959F70963079F0FB
:1016F00010F4925001C09A50923068F4803F69F023
:1017000018F4883E40F409C0843F29F406C0883E9E
:1017100020F0813F11F080E0089581E00895FC0100
:10172000808191810E94610D0E94740B0895CF9376
:10173000DF9300D000D01F92CDB7DEB70F900F908F
:101740000F900F900F90DF91CF910895CF93DF937B
:1017500000D000D000D0CDB7DEB726960FB6F894F3
:10176000DEBF0FBECDBFDF91CF91089508950895DC
:101770000C94B70B0C94B80B0E94BA0B6093D30176
:101780007093D4018093D5019093D6010C94580B9B
:101790000C94BC0B0F931F930091D3011091D401B3
:1017A0002091D5013091D601602B712B822B932B88
:1017B0001F910F910C94BC0B0F931F930091D301B9
:1017C0001091D4012091D5013091D601602371236D
:1017D000822393231F910F910C94BC0B0F931F93A3
:1017E0000091D3011091D4012091D5013091D601FF
:1017F00060277127822793271F910F910C94BC0BB0
:101800000C941A050E94000C6093CF017093D001D4
:101810008093D1019093D2010C94580B60E070E05A
:10182000CB010C94020C0F931F9341E050E060E059
:1018300070E08A019B0104C0000F111F221F331F9B
:101840008A95D2F7C901B8011F910F910C94020C2F
:101850000F931F9341E050E060E070E004C0440F3C
:10186000551F661F771F8A95D2F78091CF019091FF
:10187000D001A091D101B091D2018A019B01082B26
:10188000192B2A2B3B2BC901B8011F910F910C94E6
:10189000020C0F931F9341E050E060E070E004C041
:1018A000440F551F661F771F8A95D2F740955095B4
:1018B000609570958091CF019091D001A091D10158
:1018C000B091D2018A019B01082319232A233B23CB
:1018D000C901B8011F910F910C94020C0F931F9333
:1018E00041E050E060E070E004C0440F551F661F07
:1018F000771F8A95D2F78091CF019091D001A09166
:10190000D101B091D2018A019B01082719272A270A
:101910003B27C901B8011F910F910C94020C0F9342
:101920001F930091CF011091D0012091D1013091EE
:10193000D201602B712B822B932B1F910F910C9452
:10194000020C0F931F930091CF011091D0012091B1
:10195000D1013091D20160237123822393231F91FF
:101960000F910C94020C0F931F930091CF011091D3
:10197000D0012091D1013091D201602771278227B7
:1019800093271F910F910C94020C0895292F220F79
:10199000920F990F890FE82FE695E695E6958770E7
:1019A00051E001C0550F8A95EAF785E0E89FF00104
:1019B0001124E856FE4F20E030E070E04081CB017A
:1019C000022E02C0969587950A94E2F78170819560
:1019D00084278523842781932F5F3F4F253031054E
:1019E00069F70895292F220F920F990F890F682FF9
:1019F000669566956695982F977085E0689FB0010B
:101A0000112440E050E080E0FB01E40FF51FE856B0
:101A1000FE4F208130E0092E02C0369527950A94AA
:101A2000E2F721703327042E01C0220F0A94EAF74F
:101A3000822B4F5F5F4F4530510531F70895BF92BC
:101A4000CF92DF92EF92FF920F931F93CF93DF938A
:101A50008C01C090CF01D090D001E090D101F090E6
:101A6000D2018091D3019091D401A091D501B09180
:101A7000D601C82AD92AEA2AFB2ACFE1D0E0D70129
:101A8000C6010C2E04C0B695A795979587950A9424
:101A9000D2F780FD04C0219790F7B12C07C0BC2E6F
:101AA000B8018C2F0E9448140197A9F38B2DDF9168
:101AB000CF911F910F91FF90EF90DF90CF90BF904B
:101AC0000895CF93DF93EC010E941F0DBE010E9489
:101AD0004814DF91CF9108951F93CF93DF93EB01CB
:101AE00090919701992321F0CB010E94610D13C0C1
:101AF000882349F0CB010E941F0D182F682FCE01BB
:101B00000E94C60C04C0CB010E94F20C182FBE012B
:101B1000812F0E944814DF91CF911F9108951F9348
:101B2000CF93DF93C091D70116E08091D801C817F9
:101B300099F0D0E01C9FF0011D9FF00D1124E75299
:101B4000FE4F4081518162817381848195810E9421
:101B5000A60B2196C770E9CFDF91CF911F91089511
:101B60004091090250910A0260910B0270910C029F
:101B700080910D0290910E020C94A60BEF92FF92B1
:101B80000F931F93CF93DF9380910E0282958F70F6
:101B900009F065C080910B02882309F460C0809130
:101BA000D701F090D8011091090200910A026091CA
:101BB0000C0270910D0291E01F3F09F090E0C0917E
:101BC0000801D0910901292F96E0E92E8F1509F41B
:101BD00046C06115710521F00F3F21F030E003C0D0
:101BE00031E001C0322F90E030FD36C0E89EF001B8
:101BF000E99EF00D1124DF01A752BE4F11963C91D2
:101C00001197301329C03C91311326C012963C9194
:101C10001297311121C013964D915C911497461B78
:101C2000570B4C175D07C0F480910E028F708061D6
:101C300080930E02E252FE4F80818F70806180831C
:101C400089E092E00E94240BDF91CF911F910F91C8
:101C5000FF90EF900C948F0D01968770B7CFDF91B6
:101C6000CF911F910F91FF90EF9008959F92AF92A7
:101C7000BF92CF92DF92EF92FF920F931F93CF9379
:101C8000DF93CDB7DEB761970FB6F894DEBF0FBE16
:101C9000CDBF8C0185E0F801DE011D9601900D920B
:101CA0008A95E1F7D8011296EC9090910902E091A3
:101CB0000A0220910C0230910D022115310531F0FC
:101CC000EF3F31F481E09F3F19F403C081E001C090
:101CD00080E0B82FB1709B2E80FD47C1D8014C9198
:101CE00011965C9111971396AD90BC90149789E072
:101CF000C82E82E0D82EF0900B02B501621B730B48
:101D00002091080130910901FF2009F4D9C0809188
:101D10000E026217730708F095C0282F207F09F084
:101D200052C05E1313C0491311C0FE2CE1100EC047
:101D30008F70806180930E020E94B00DC6010E94D8
:101D4000240B80910E02F80185834DC1AB2831F040
:101D50005F3F31F481E04F3F19F403C081E001C0DF
:101D600080E080FD03C081E08E2502C080E090E02D
:101D7000F82FF170FF2E80FF1CC08091D7012091B9
:101D8000D80136E0821709F40BC190E0389FF001CA
:101D9000399FF00D1124E752FE4F6181561306C0A2
:101DA0006081461303C06281E61203C0019687700A
:101DB000E9CFFE2CEE2009F416C180910E0281605D
:101DC00080930E0254C05E1306C0491304C0E11094
:101DD00002C0F80199C0C8010E948F0B882361F1ED
:101DE000EE2051F120910E02822F82958F7090E0AB
:101DF000029774F08091090290910A0298878F836C
:101E00001986BB86AA862C87CE0107960E94240BD2
:101E100086E0F801A9E0B2E001900D928A95E1F721
:101E20000E94BE0D0E94B00D0AC05E1711F1C801DC
:101E30000E948F0B81112CC0C8010E94240BFF242B
:101E4000F394D1C0282F207F81F77A2DB98AA88AF0
:101E50006E2D89890E94970B89E092E00E94240BE5
:101E600086E0D6011D928A95E9F70E94B00DF12C0B
:101E7000BAC04913DCCFE110DACFF8018583C8017D
:101E80000E94240B86E0D6011D928A95E9F7ABC02B
:101E9000EE2091F220910E02822F82958F7090E0B9
:101EA00002970CF4B5CF8091090290910A029A83AF
:101EB00089831B82BD82AC822E83CE010196A6CF80
:101EC0006217730708F044C0FE2CEE2009F4B4CF6B
:101ED0005E1330C049132EC020910E0220FD21C098
:101EE000822F82958F70482F50E041155105C9F01F
:101EF000F80125834F30510541F08F5F982F92955F
:101F0000907F822F8F70892B8583C8010E94240BBC
:101F100086E0F801A9E0B2E001900D928A95E1F720
:101F20003CC086E0F801A9E0B2E001900D928A95EC
:101F3000E1F759C0C8010E948F0B811169CF8091D0
:101F40000E02816080930E02C8010E94240B4BC0D8
:101F50007A2DB98AA88A6E2D89890E94970B86E00E
:101F6000D6011D928A95E9F718C0EE2009F464CFD6
:101F7000C8010E948F0BF82E882309F45DCF86E0FC
:101F8000F801A9E0B2E001900D928A95E1F789E0AD
:101F900092E00E949D070E94BE0D0E94B00D23C0DA
:101FA0004D875E878D859E850E94610D292F229524
:101FB0002F70223028F49F7039F0811105C00BC0BA
:101FC000243028F49F7049F4805E883020F0C801E6
:101FD0000E94240B9F2CF92C06C0D80115969C91C9
:101FE000907F91F7F8CF8F2D61960FB6F894DEBFF2
:101FF0000FBECDBFDF91CF911F910F91FF90EF905A
:10200000DF90CF90BF90AF909F9008951F93CF9394
:10201000DF93CDB7DEB72C970FB6F894DEBF0FBEB7
:10202000CDBF4F83588769877A878B879C87CE017E
:1020300007960E94360E8823D1F09F8188852A85D5
:102040003B85232B31F08F3F31F481E09F3F19F422
:1020500003C081E001C080E080FD47C04F8158850A
:1020600069857A858B859C850E94A60B3EC086E09B
:10207000FE013796DE01119601900D928A95E1F7E7
:10208000FF81E8856A857B856115710531F0EF3F39
:1020900031F481E0FF3F19F403C081E001C080E02A
:1020A00080FD23C02091D80130E0C90101968770DE
:1020B00099274091D70150E084179507F1F1F983F2
:1020C000EA837D836C8396E0929FD001939FB00D4D
:1020D0001124A752BE4FFE01319601900D929A95A0
:1020E000E1F78093D8010E948F0D16E08091D7010F
:1020F0009091D801891771F1189FC001112487525E
:102100009E4F0E94360E882329F1E091D7011E9F31
:10211000F0011124E752FE4F4081518162817381A9
:10212000848195810E94A60B8091D70190E0019651
:10213000877099278093D701D9CF0E94700B109296
:10214000D8011092D701E9E0F2E086E0DF011D92AC
:102150008A95E9F72C960FB6F894DEBF0FBECDBF77
:10216000DF91CF911F91089580912F0285958595DC
:102170008595089580912F028770089590912F0280
:10218000977081E009F480E00895809152020895EB
:1021900090915202892B80935202089580959091DC
:1021A0005202892380935202089510925202089598
:1021B00090915102892B80935102089580959091BE
:1021C000510289238093510208951092510208957B
:1021D00080913002089508950C94EB100C94EC104B
:1021E0009091B30292FD08C090913002981721F0AF
:1021F000809330020C94EE10089580913002882371
:1022000029F01092300280E00C94EE100895CF93E4
:10221000DF93E0910A01F0910B01809152028083DB
:10222000E0910A01F0910B01908180915102892B7C
:10223000808380913002882381F0E0910A01F0913F
:102240000B019081892B808380910A0190910B0171
:102250000E943A1C81110E94FD10C0910A01D09188
:102260000B0140E250E06FE072E0CE010E94442694
:10227000892B69F080E2FE01AFE0B2E001900D929F
:102280008A95E1F7CE01DF91CF910C94E91BDF91A4
:10229000CF9108950C94EB109091B30292FD10C071
:1022A00098E0899F90011124262B20932F020E94F1
:1022B000280C80912F028595859585950C944A115F
:1022C0000C94280C10922F0280E00C944A1120915B
:1022D0002F028095822380932F02982F977099F474
:1022E00030E0482F082E000C550B2417350759F005
:1022F0009091B30292FD07C08595859585950E94C2
:10230000490C0C94621108959091B30292FB22271C
:1023100020F9281769F080FB92F99093B30280911D
:10232000B2029091B3020E94CC1182E00C9467112A
:1023300008958091B30282FB882780F991E0892774
:102340000C94841181E00C94841180E00C9484112D
:1023500080E090E00E945F2621E0893E9E4F09F0D8
:1023600020E0822F089582E090E00C94512683E0D3
:1023700090E00C945126CF9384E090E00E94512687
:10238000C82F82E290E00E9451262C2F30E0A90154
:10239000582BCA01CF910895CF93C92F682F84E09D
:1023A00090E00E9465266C2F82E290E0CF910C9421
:1023B00065268FE090E00C945926AB01BC018FE0BC
:1023C00090E00C947726AB01BC0183E190E00C9483
:1023D000772660E070E0CB010C94E31169EE7EEFAC
:1023E00080E090E00E94832660E082E090E00E941E
:1023F000652660E083E090E00E9465261092D3019C
:102400001092D4011092D5011092D60160E084E0C0
:1024100090E00E94652660E082E290E00E946526DE
:1024200060E085E090E00E94652660E086E090E054
:102430000E9465266FEF87E090E00E94652640E0ED
:1024400050E0BA0188E090E00E94772660E08DE0DD
:1024500090E00E94652640E050E0BA0188E190E0FB
:102460000E94772660E087E190E00E94652640E0C8
:1024700050E0BA018CE190E00E94772660E070E0C5
:1024800080E290E00E94832640E050E0BA0188E1BB
:1024900090E00E9477260C94EF040C94EE11682FC4
:1024A0008EE090E00C9465260E949D1D609365026D
:1024B0007093660280936702909368026093610252
:1024C000709362028093630290936402089585B7CB
:1024D000806885BF85B7806885BF089581E00895CD
:1024E0000C946E1208950C9472120C9419050C94AD
:1024F00072120C9477120C9472120E94671284E28A
:1025000095E10E94D31B0E947B120C9479120E94C9
:1025100073120C9472120E9427150C9437070E94B4
:10252000881D0E9457150E948B120C9475128F9271
:102530009F92AF92BF92CF92DF92EF92FF920F9352
:102540001F93CF93DF93CDB7DEB72A970FB6F894DA
:10255000DEBF0FBECDBF0E946815982E81110E946C
:10256000541283E5A82E82E0B82E00E010E0802E01
:10257000802F0E944B15D82EF501C1905F01C8260F
:10258000B1F40F5F1F4F0E30110589F78FEF89836C
:102590008A831B820E94911D8160782F9D838C838A
:1025A00049815A816B818D810E9453072FC0809190
:1025B000690281FD0E945115E12CFF24F3948C2DBA
:1025C0008F21F1F00E947012882399F0EE828F82A1
:1025D000DF2081E009F480E088870E94911D8160FE
:1025E000782F9A8789874E815F8168858A850E94C6
:1025F0005307F801ED5AFD4F8081F826F08206C09E
:10260000E394FF0CF6E0EF12DACFBBCF81E091103C
:1026100001C080E02A960FB6F894DEBF0FBECDBF92
:10262000DF91CF911F910F91FF90EF90DF90CF90AE
:10263000BF90AF909F908F9008950E9497120E9434
:1026400095170C944807CF93DF930E944D14EC012B
:10265000811521E5920708F045C0811530E5930703
:1026600008F094C0883E910528F5803E910508F059
:10267000F8C0883A910570F4853A910508F07CC05D
:102680008130910509F475C008F4E8C0049708F09A
:10269000E8C0E4C08F3B910508F0E0C0C85AD0E024
:1026A000CC0FDD1FCF5ADE4F0990D881C02DCE014F
:1026B0009464D8C0811540E2940758F4811551E024
:1026C000950708F0CEC08D3E910508F4C7C090650F
:1026D000C9C0C11580E4D80708F4C0C0DF70CE01BE
:1026E000906AC0C0811525E59207A8F4811534E5EC
:1026F000930708F095C0811543E5940708F07BC067
:10270000811552E5950708F061C0D82FCC27CE017E
:10271000816F906AA7C0C11589E5D807A0F4C115DB
:1027200028E5D20708F082C0C11536E5D30708F0C6
:1027300095C08C2F0E94E1148F7190E0D82FCC2788
:10274000CE0190628FC0C1154AE5D40708F474C069
:10275000CE0190568115904208F080C08D2F8F7168
:102760000E94E114DD27D0628F71AE01582BCA019F
:1027700079C081E090E076C0C55AD0E0C158DE4F04
:102780008881C82FD0E0CE0190646CC074E096952B
:1027900087957A95E1F7282F23703C2F337081E0DD
:1027A00090E002C0880F991F3A95E2F79C68AC014F
:1027B000522B9A019C2F9F709695969550E2959F6B
:1027C000E0011124C9018C2B9D2B4CC083709927EB
:1027D00021E030E002C0220F331F8A95E2F79C2FE0
:1027E0009695969580E2989FE0011124C22BD32BF9
:1027F000CE019C6837C08370992721E030E002C089
:10280000220F331F8A95E2F79C2F9695969540E20A
:10281000949FE0011124C22BD32BCE019A6822C0D1
:10282000D82FCC27CE01846F906A1CC0DC2FCC2718
:10283000CE01806F906A16C08C2F8F700E94E114B9
:1028400094E0D695C7959A95E1F7CF70D0E0DC2F4C
:10285000CC27D0699E01282BC90104C080E090E0FC
:1028600001C0CE01DF91CF91089524E5829FC00180
:102870001124FC0126E0729FE00DF11D1124E60FEA
:10288000F11DEE0FFF1FE45EFE4F859194910895B8
:102890000E9435140E94231308958238910569F12E
:1028A000B0F48133910509F46DC048F48932910583
:1028B00009F463C08A32910509F469C0089585332B
:1028C000910509F455C089339105B9F00895833E07
:1028D000910569F138F4803E9105B1F0823E910591
:1028E00009F10895863E9105A9F1873E9105B9F158
:1028F000843E910509F064C023C02091B20220FDFE
:102900004FC021FD4DC008958091B20280FD44C0AA
:102910008091B30280FF44C08091B20284FD42C026
:1029200083EE4DC08091B20282FF38C0F5CF809116
:10293000B20282FD33C08091B30280FD31C0ECCF82
:102940008091B30281FF32C08091B20284FD2AC01F
:1029500087EE35C08091B20283FF26C0F5CF80910B
:10296000B20283FD21C08091B30281FD1FC0ECCF74
:102970008091B20285FD1CC01DC08091B20285FD10
:1029800019C016C08091B20286FD16C017C0809192
:10299000B20286FD13C010C089E311C082EE0FC0E1
:1029A00080EE0DC080E00BC086EE09C084EE07C04B
:1029B00089E205C085E303C08AE201C081E390E0BB
:1029C00008959091B20292FF0DC0282F28712830EF
:1029D00019F4877F846006C0282F2471243011F4F5
:1029E0008B7F886093FF0DC0282F2871283119F440
:1029F000877E846106C0282F2471243111F48B7ED8
:102A000088612091B30220FF0DC0382F3871383013
:102A100019F4877F816006C0382F3171313011F48D
:102A20008E7F886021FF0DC0282F2871283119F46E
:102A3000877E816106C0282F2171213111F48E7E9D
:102A4000886194FD877E089580E0089508950E942E
:102A5000A811811102C00E944D120E94B3118093EF
:102A600069020E94BB119093B3028093B2020E944C
:102A700026150E94B711682F70E080E090E00E9458
:102A8000C80B6091CF017091D0018091D1019091DC
:102A9000D2010C94000CE82FF0E0EE53FD4F808142
:102AA0000895089508950C9452150C9452150E949F
:102AB0007803E4EBF2E0A2ECB2E011921D9282E026
:102AC000E23CF807D1F78EE00E947B150C949C0540
:102AD000CF9384EB92E00E948303C82F282F4EE00F
:102AE00062EC72E084EB92E00E948E150E949E05DB
:102AF0008C2FCF910895CF93C82F90E00E9423256B
:102B000080936D0290936E02282FFC018E2F821B02
:102B10008C1710F41192FACFCF910895DF92EF92B3
:102B2000FF920F931F93CF93DF93082FF92EE62E7A
:102B3000D72E142FD22FC0916A02CC23C9F10E9444
:102B4000911D20916B0230916C02AC01421B530B22
:102B50009A0190936C0280936B024F3F510509F0EC
:102B600020F4452B09F454C002C02FEF30E010923E
:102B70006A0210926F0240916D02E42FF0916E0292
:102B800090E030E08E2F841B811768F480818823C9
:102B900041F0281718F010829C2F03C0821B8083FD
:102BA0003C2F3196EFCF30936A0290936F0230C082
:102BB000222331F10E94911D90936C0280936B024D
:102BC00090916D0280916A02AE2DBD2DC02FDF2D38
:102BD000E92FF0916E023EE12E2F291B211768F498
:102BE00029914C91421731F04081411103C030834B
:102BF0002C9381E031961196EFCF80936A020CC03E
:102C000080E090916F02992339F08111D9CFD2CF12
:102C1000D111D6CF81E0F5CFDF91CF911F910F91E8
:102C2000FF90EF90DF9008950E94BE1F0E948F12C8
:102C30000C94CA1F0E94CE1F0E941D130C94E81F03
:102C40000E942F1D0E94A51F0E947D120E94141633
:102C50000E941A160E948712FBCF8091770280FF94
:102C600006C06091110170E0660F771F26C081FFDA
:102C700004C06091110184E005C082FF07C060912B
:102C8000110188E0689FB001112417C0909176026D
:102C90009923D1F060911001961788F720911101C6
:102CA00088E0289F90011124929FA001939F500DCE
:102CB000112470E0CA010E9409256038710540F4B2
:102CC0006115710519F406C068E070E0862F08955B
:102CD0008FE7089581E008958091770280FF08C012
:102CE00060910D0170E0759567957595679521C0A8
:102CF00081FF06C060910D0170E07595679519C060
:102D000082FF04C060910D0170E010C090917502C7
:102D1000992399F060910C019617A0F780910D010D
:102D2000899FC001112470E00E9409256038710557
:102D300040F46115710519F406C061E070E0862F5A
:102D400008958FE7089581E008958D3E21F40E9453
:102D50002D16819504C08E3E29F40E942D16809375
:102D60007A0208958F3E21F40E942D16819504C0A9
:102D7000803F29F40E942D16809379020895893F9F
:102D800019F40E946C1605C08A3F31F40E946C163B
:102D9000819580937B0208958B3F21F40E946C16ED
:102DA000819504C08C3F29F40E946C1680937C02AC
:102DB00008959FE0980F983078F421E030E0A90161
:102DC00002C0440F551F9A95E2F7CA01909178020C
:102DD000892B8093780208958D3F21F480917702AA
:102DE00081600BC08E3F21F480917702826005C024
:102DF0008F3F29F480917702846080937702089551
:102E00008D3E39F490917A0297FF35C010927A0284
:102E100059C08E3E29F490917A021916BCF32BC04A
:102E2000909179028F3E29F497FF25C01092790284
:102E300049C0803F19F41916CCF31DC090917B0254
:102E4000893F29F41916BCF410927B023BC08A3FDB
:102E500019F497FF10C0F8CF8B3F39F490917C02A2
:102E600097FF09C010927C022DC08C3F21F49091F5
:102E70007C021916BCF39FE0980F983080F421E093
:102E800030E0A90102C0440F551F9A95E2F7CA012C
:102E900080959091780289238093780213C08D3FAA
:102EA00021F4809177028E7F0BC08E3F21F48091B8
:102EB00077028D7F05C08F3F29F4809177028B7F49
:102EC0008093770280917902811106C080917A0205
:102ED000811102C01092760280917B02811106C09E
:102EE00080917C02811102C01092750208950E94A7
:102EF000911D20917902211104C020917A02222390
:102F000021F0909374028093730220917B0221112F
:102F100004C020917C02222321F0909372028093BE
:102F2000710288E792E00C94031CEF92FF920F93DA
:102F30001F93CF93DF9300D000D01F92CDB7DEB7A1
:102F400085E0E8E7F2E0DE01119601900D928A95A6
:102F5000E1F7E0907902F0907A0200917B02109103
:102F60007C021092790210927A0210927B021092E7
:102F70007C02E11003C0FF2009F45DC08091730260
:102F8000909174020E94A91DAC0190917602992340
:102F900039F02091120130E02417350758F04BC06A
:102FA000209170028AE0289F900111242417350790
:102FB00018F041C09F3F19F09F5F90937602EE207A
:102FC00061F00E942D161E1414F09FEF01C091E0D5
:102FD000989F902D112490937902FF2061F00E9418
:102FE0002D161F1414F09FEF01C091E0989F902DB3
:102FF000112490937A02309179023323E1F02091E9
:103000007A022223C1F045EB3403C0011124992335
:1030100019F09093790203C081E08093790235EB37
:103020002303C0011124992319F090937A0203C05D
:1030300081E080937A02011103C0112309F45DC07D
:1030400080917102909172020E94A91DAC01909131
:103050007502992339F020910E0130E024173507CD
:1030600058F04BC020910F018AE0289F9001112455
:103070002417350718F041C09F3F19F09F5F9093C8
:103080007502002361F00E946C16101614F09FEF79
:1030900001C091E0989F902D112490937B02112301
:1030A00061F00E946C16111614F09FEF01C091E0C0
:1030B000989F902D112490937C0230917B023323B2
:1030C000E1F020917C022223C1F045EB3403C001E2
:1030D0001124992319F090937B0203C081E080931F
:1030E0007B0235EB2303C0011124992319F090933F
:1030F0007C0203C081E080937C028091790281117F
:103100000BC080917A02811107C080917B028111EE
:1031100003C080917C0281110E947717EA82FB82B2
:103120000C831D8385E0FE013196A8E7B2E0019093
:103130000D928A95E1F70F900F900F900F900F90DE
:10314000DF91CF911F910F91FF90EF900895E8E7E5
:10315000F2E085E0DF011D928A95E9F71092760290
:1031600010927502109277020895CF93DF93EC01CD
:10317000FB018281882309F43CC1C430FDE5DF07EF
:1031800060F4CB3F9CE5D90788F49E0122503C4572
:103190002431310508F02EC109C0C236EDE5DE0745
:1031A00029F0C63AFDE5DF0709F024C10E94BB11F2
:1031B0009093B3028093B202C1318CE5D80709F431
:1031C000C6C008F042C0C930ECE5DE0709F49BC078
:1031D00000F5C5308CE5D80709F485C078F4C33014
:1031E000ECE5DE0709F478C008F07AC0C230DC45AF
:1031F00009F0F5C08091B2028160EFC0C7309CE554
:10320000D90709F478C008F07AC08091B2028061D1
:10321000E4C0CD30FCE5DF0709F487C058F4CB30BB
:103220009CE5D90709F479C008F07BC08091B2020F
:1032300088606FC0CF30FCE5DF0709F480C008F07C
:1032400082C08091B202877FC8C0CE3F9CE5D9077B
:1032500009F471C000F5C531FCE5DF0709F485C04C
:1032600068F4C3319CE5D90709F475C008F095C02E
:103270000E94700B8091B2028F77AFC0CC3FFCE50B
:10328000DF07A9F108F054C0CB3FDC4509F0A7C027
:103290008091B30240C0C230EDE5DE0709F489C079
:1032A00058F4C1158DE5D80709F45AC008F069C073
:1032B0008091B30282602FC0C236EDE5DE0709F4CB
:1032C0007CC0C63AFDE5DF0709F481C0C330DD45A7
:1032D00009F085C080E06EC08091B20282607DC03E
:1032E0008091B20216C08091B202886076C080914F
:1032F000B30282604FC08091B20280626EC0809142
:10330000B20280646AC00E94700B8091B202806831
:1033100064C0846062C081603DC08091B2028E7FD3
:103320005CC08091B2028D7F58C08091B20216C0FD
:103330008091B30218C08091B3028D7F2BC0809121
:10334000B2028F7E4AC08091B2028F7D46C08091CA
:10335000B2028F7B42C08091B202877F8B7F3DC0DB
:103360008091B3028D7F8E7F15C08091B20282FB67
:10337000222720F991E0922790FB82F990FB83F9B4
:103380002CC08091B302982F909591708E7F892BDD
:1033900090FB81F98093B30222C00E94700B809150
:1033A000B20287FB222720F991E0922790FB87F950
:1033B00014C081E00E944F1212C08091B20284FBBF
:1033C000222720F991E0922790FB84F906C0809192
:1033D000B202982F909590FB80F98093B202809171
:1033E000B2029091B3020E94CC110E94700B80E057
:1033F00001C081E0DF91CF910895CF93DF938631B3
:103400009C4541F5EB010E94C510982F8A812091BF
:103410000A0130910B01882379F09A7A81E009F44E
:1034200080E080937D02911102C069E201C065E3F2
:10343000C9010E94D01C0AC080917D02811102C086
:1034400069E201C065E3C9010E94DB1C0E9407110B
:1034500080E001C081E0DF91CF9108950F931F9329
:10346000CF93DF93C42FD22FFC0182818823C9F030
:10347000409380020E94911D90937F0280937E0270
:1034800080E28C0F883008F057C0C77081E001C01F
:10349000880FCA95EAF7DF91CF911F910F910C9495
:1034A000D50880918002481330C080917E029091AF
:1034B0007F020E94A91D883C910538F510E21D0F7E
:1034C000CD17B9F080E28C0F883040F4C77081E0EE
:1034D00001C0880FCA95EAF70E94DC08183028F569
:1034E00081E09D2F977001C0880F9A95EAF70E949E
:1034F000D508802F0E94CC081830F0F4D77081E0F6
:1035000001C0880FDA95EAF70AC080E28C0F883094
:1035100098F4C77081E001C0880FCA95EAF7DF917F
:10352000CF911F910F910C94DC08802FDF91CF91E8
:103530001F910F910C94CC08DF91CF911F910F91A7
:1035400008950F939C01CB01243F4CE5340731F1E2
:1035500088F4293DFCE53F07D9F02A3D4CE53407C6
:1035600079F1283D3C45A9F506E221EE41EE68EDF2
:103570007CE52BC0263FFCE53F07E1F0A8F0273FA4
:103580003C4539F507E225EE46EE67EF7CE51DC0C8
:1035900007E225EE45EE69ED7CE517C006E221EE77
:1035A00040EE64EF7CE511C007E225EE44EE65EFE6
:1035B0007CE50BC006E221EE42EE66EF7CE505C03D
:1035C00008E221E045EE6AED7CE50E942E1A80E0DB
:1035D00008C0FC018281882319F01092800201C08A
:1035E00081E00F9108951092B9008CE08093B800AB
:1035F00008959F92AF92BF92CF92DF92EF92FF9287
:103600000F931F93CF93DF93B82EEB010E94911D70
:103610006C01C431D10558F0CF3F8FEFD80759F076
:10362000CE0164E170E00E94F5247B0107C0EE2426
:10363000E394F12C03C025E0E22EF12C84E8A82EBF
:1036400094EA992E1092BC009092BC000E94911DA9
:103650008C018091BC0087FD08C00E94911D801BD9
:10366000910B8E159F05A8F32AC08091B900887F21
:10367000883041F08091B900887F803119F00FEFD8
:103680001FEF1FC0B092BB00A092BC000E94911D12
:103690008C018091BC0087FD08C00E94911D801B99
:1036A000910B8E159F05A8F30AC08091B900887F01
:1036B000883111F0803419F700E010E00EC00EEFF1
:1036C0001FEFCF3F8FEFD80709F4BCCFC6010E9490
:1036D000A91D8C179D0708F4B5CFC801DF91CF91C4
:1036E0001F910F91FF90EF90DF90CF90BF90AF9020
:1036F0009F9008950F931F93CF93DF93EB018093D7
:10370000BB0084E88093BC000E94911D8C018091D5
:10371000BC0087FD0EC0CF3F8FEFD807C1F30E94DA
:10372000911D801B910B8C179D0788F38EEF9FEFE7
:103730000CC02091B900287F81E090E0283211F47C
:1037400080E090E0919581959109DF91CF911F9153
:103750000F9108950F931F93CF93DF93EC0184E8AB
:103760008093BC000E94911D8C018091BC0087FD5C
:103770000EC0CF3F8FEFD807C1F30E94911D801B71
:10378000910B8C179D0788F38EEF9FEF03C08091FC
:10379000BB0090E0DF91CF911F910F91089584E9D4
:1037A0008093BC00089590939301809392010895B3
:1037B00090938602809385020895E0918502F091AE
:1037C0008602309721F00190F081E02D099480E08D
:1037D0000895E0918502F0918602309799F020914A
:1037E0001F01222359F02091B20227FF07C0DC01FC
:1037F0002C9111962C93119726E02C930280F38143
:10380000E02D09940895E0918502F09186023097A9
:1038100021F00480F581E02D099408952091830220
:10382000309184022817390771F0909384028093B5
:103830008302E0918502F0918602309721F00680A4
:10384000F781E02D09940895209181023091820240
:103850002817390771F09093820280938102E091DA
:103860008502F0918602309721F00084F185E02DE9
:1038700009940895FC01329680911F01882331F04C
:103880008091B20287FF02C09EE101C096E080E015
:10389000915028F021912223D9F38F5FF9CF089519
:1038A000662351F120911F012223E9F02091B202F9
:1038B00027FF19C0462F4695469546954E31E0F4B0
:1038C000677021E030E002C0220F331F6A95E2F7F3
:1038D000FC01E40FF11D828190E02823392381E06F
:1038E000232B69F409C0FC013296089621916217D6
:1038F00029F0E817F907D1F780E0089581E00895ED
:103900009C01FC0132969FEF80E04191461789F0BF
:103910009F3F19F4411101C0982F8F5F8630A9F79E
:103920009F3F39F0F901E90FF11D97FDFA95628388
:10393000089508959C012A5F3F4FFC014281461380
:1039400001C01282019682179307B9F70895262FB6
:103950002695269526952E3168F4FC01E20FF11D7F
:10396000677021E030E001C0220F6A95EAF782819A
:10397000282B22830895262F2695269526952E31CD
:1039800070F4FC01E20FF11D677021E030E001C02E
:10399000220F6A95EAF720958281282322830895D1
:1039A00020911F01222329F02091B20227FD0C94BF
:1039B000A71C0C94801C20911F01222329F0209128
:1039C000B20227FD0C94BB1C0C949A1C20911F0181
:1039D000FC013296222331F08091B20287FF02C0AF
:1039E0008EE101C086E0DF011D928A95E9F7089516
:1039F00008950C94F81C83E0809387020C94F91CC2
:103A0000811102C081E001C082E0809387020C94A2
:103A1000F91C0C94001D81E0809387020C94F91C22
:103A20000C940B1D08950C94121D0C94131D0C94F2
:103A3000121D0C94121DCF930E94D7030E9468158B
:103A40000E94171DC0E08C2F0E944B15811104C0ED
:103A5000CF5FCE30C1F701C081E0CF9108950895C6
:103A60001F920F920FB60F9211248F939F93AF93D3
:103A7000BF9380918802811113C08091D0029091F0
:103A8000D102A091D202B091D3024196A11DB11DE5
:103A90008093D0029093D102A093D202B093D3022C
:103AA000BF91AF919F918F910F900FBE0F901F907C
:103AB00018958091D802843031F10E94020610924C
:103AC000880220E488E190E00FB6F894A8958093EE
:103AD00060000FBE2093600083B7817F846083BF46
:103AE00083B7816083BF7894889583B78E7F83BFC7
:103AF0000FB6F894A895809160008861809360006B
:103B0000109260000FBE08950E94700B0C94060680
:103B100082E084BD93E095BD9AEF97BD80936E00DF
:103B200008952FB7F8948091D0029091D102A0917E
:103B3000D202B091D3022FBF08952FB7F8946091AD
:103B4000D0027091D1028091D2029091D3022FBF06
:103B500008959C014FB7F8948091D0029091D102C2
:103B6000A091D202B091D3024FBF821B930B089554
:103B700078941F920F920FB60F9211248F939F93F8
:103B8000AF93BF938091D0029091D102A091D202C5
:103B9000B091D3020196A11DB11D8093D0029093E4
:103BA000D102A093D202B093D302BF91AF919F9163
:103BB0008F910F900FBE0F901F901895F89481E091
:103BC0008093E00080E28093D800E9ECF0E010827E
:103BD0008FE19EE40197F1F700C000001DBA10923A
:103BE00068001CBC10BE1FBA10927A0010926E00C2
:103BF00010926F0010927100109272001082ECEB24
:103C0000F0E0108214B817B81AB81DB810BA1082B4
:103C100015B818B81BB81EB811BA0C94003F089517
:103C20008091AC020895089522E02093E9002FEFDF
:103C30003091E800215035FD06C035ED3A95F1F799
:103C400000002111F5CF2091E80025FF0BC040E0D6
:103C500050E065E070E00E9457208091E8008E7788
:103C60008093E8000895CF93DF9320911F012223D2
:103C700039F02091B20227FF03C060E223E002C0C6
:103C800068E021E02093E9002FEF3091E800215017
:103C900035FD06C035ED3A95F1F700002111F5CF5D
:103CA0002091E80025FF1DC0EC0180911F018111CA
:103CB00005C040E050E068E070E003C070E040E024
:103CC00050E0CE010E9457208091E8008E778093CB
:103CD000E80080E2FE01ACE8B2E001900D928A9526
:103CE000E1F7DF91CF9108958093890270938B0261
:103CF00060938A028091D802843001F583E080933A
:103D0000E9008FEF9091E800815095FD06C095ED98
:103D10009A95F1F700008111F5CF8091E80085FFB9
:103D20000DC040E050E063E070E089E892E00E945E
:103D300057208091E8008E778093E8000895BC01B9
:103D400084E00C94741EBC0183E00C94741E80917A
:103D5000D702811109C00E94E8210E94452280916A
:103D6000E20084608093E20008951092D7020895E3
:103D70000C94101D6091D40281E0611101C080E0BB
:103D80000C94FB1C9091D80281E0943009F080E003
:103D90006091D4020C94001D42E061EC81E00E942D
:103DA000612142E061EC82E00E94612142E261EC2B
:103DB00083E00E9461219091D80281E0943009F063
:103DC00080E06091D4020C94091D8091DA02833066
:103DD00009F463C030F4813071F0823009F49CC082
:103DE00008958A3009F488C08B3009F46EC0893098
:103DF00009F0AAC020C08091D902813A09F0A4C07C
:103E00008091E800877F8093E8008091DD029091A7
:103E1000DE02892B21F460E28CE892E003C060E0CE
:103E200080E090E070E00E94A2208091E8008B7713
:103E30008093E80008958091D902813209F084C00E
:103E40008091DD029091DE02009719F0029709F04F
:103E50007BC08091E800877F8093E8008091E80034
:103E600082FD05C08091D8028111F8CF6DC02091EC
:103E7000F3008091F20090E0922B029731F4809150
:103E8000F100813011F0863021F48091F1008093AF
:103E9000AC028091E8008B7753C08091D902813ABF
:103EA00009F052C08091DD029091DE02892B09F069
:103EB0004BC08091E800877F8093E8008091E80004
:103EC00080FFFCCF80911F0136C08091D9028132E2
:103ED000D9F58091DD029091DE02892BA9F58091C0
:103EE000E800877F8093E8000E9496218091DB02A2
:103EF00080931F010C94700B8091D902813221F5BF
:103F00008091E800877F8093E8000E94962180914D
:103F1000DC028093AD0208958091D902813AA1F428
:103F20008091E800877F8093E8008091E80080FF1F
:103F3000FCCF8091AD028093F1008091E8008E77F4
:103F40008093E8000C949621089584B7877F84BFFE
:103F50000FB6F894A8958091600088618093600006
:103F6000109260000FBE90E080E80FB6F894809346
:103F70006100909361000FBE0C940B1D0E94E8211C
:103F80000E944522E2EEF0E0808184608083789494
:103F90000C94DA2483E191E00C94D81B8091D80230
:103FA0008530A9F48091D802853079F40E94591D9A
:103FB0008091D6028823B1F30E941B1D882391F3C0
:103FC0000E9441200E94700BEDCF0C94841D089537
:103FD00008950C94EB1F292F332723303105C9F0A6
:103FE00060F42130310581F02230310509F041C003
:103FF00084E590E02AE034E040C021323105E1F070
:104000002232310531F135C082E190E02EE534E015
:1040100034C099278130910549F028F0029749F57D
:10402000E4ECF3E005C0E6E0F4E002C0ECEDF3E020
:10403000849190E09F0121C063307105D0F4660F38
:10404000771FFB01E557FE4F2081318189E090E029
:1040500014C06330710568F4FB01EE0FFF1FEB57CE
:10406000FE4F20813181FB01EE57FE4F808190E0B1
:1040700004C080E090E020E030E0FA01318320834A
:10408000089580E189BD82E189BD09B400FEFDCFBC
:104090008091D8008F7D8093D8008091E00082606D
:1040A0008093E0008091E00081FDFCCF0895CF92E5
:1040B000DF92EF92FF920F931F93CF93DF93EC0168
:1040C0008B017A010E94B521811133C0E114F10402
:1040D00039F0F70180819181081B190BC80FD91F96
:1040E000C12CD12C0115110519F18091E80085FD35
:1040F00016C08091E8008E778093E800E114F10407
:1041000049F0F70180819181C80ED91ED182C08209
:1041100085E00FC00E94B521882321F30AC0899150
:104120008093F10001501109FFEFCF1ADF0ADACFB7
:1041300080E0DF91CF911F910F91FF90EF90DF9082
:10414000CF9008952091DF023091E00226173707C3
:1041500048F06115710539F42091E8002E7720931D
:10416000E80001C0B901FC0120E06115710579F199
:104170008091D8028823F1F18530F1F18091E80037
:1041800083FD3CC08091E80082FD2EC08091E80054
:1041900080FFEBCF2091F3008091F20090E0922B12
:1041A0006115710551F08830910538F42191209303
:1041B000F100615071090196F3CF21E0089709F0F1
:1041C00020E08091E8008E778093E800CECF211127
:1041D000CFCF0AC08091D802882361F0853061F08A
:1041E0008091E80083FD0AC08091E80082FFF2CF51
:1041F00080E0089582E0089583E0089581E00895C5
:104200002091DF023091E0022617370748F0611550
:10421000710539F42091E8002E772093E80001C061
:10422000B901FC0120E06115710591F18091D8027E
:10423000882309F440C0853009F43FC08091E8002C
:1042400083FD3DC08091E80082FD2FC08091E80091
:1042500080FFE9CF2091F3008091F20090E0922B53
:104260006115710559F08830910540F4249120932F
:10427000F1003196615071090196F2CF21E0089763
:1042800009F020E08091E8008E778093E800CBCFA2
:104290002111CCCF0AC08091D802882361F08530EB
:1042A00061F08091E80083FD0AC08091E80082FF00
:1042B000F2CF80E0089582E0089583E0089581E0E0
:1042C0000895982F973068F59093E900981739F082
:1042D0007091EC002091ED005091F00003C0242F6C
:1042E000762F50E021FD02C09F5FECCF3091EB00B4
:1042F0003E7F3093EB003091ED003D7F3093ED0039
:104300003091EB0031603093EB007093EC00209320
:10431000ED005093F0002091EE0027FDE5CF80E006
:1043200008958F708093E90081E008958091D9020B
:1043300087FF11C08091E80082FD05C08091D802FE
:104340008111F8CF11C08091E8008B770BC080916C
:10435000D802882349F08091E80080FFF8CF80914F
:10436000E8008E778093E80008952091E400309172
:10437000E50095E64091EC00842F817040FF23C05A
:104380008091E80080FD1DC08091D802882399F0BB
:10439000853099F08091EB0085FD11C04091E400DB
:1043A0005091E5002417350729F3915011F09A0137
:1043B000E1CF84E0089582E0089583E0089581E0EC
:1043C000089580E008954091E80042FFDDCF089510
:1043D0000E9456220E945E22E0EEF0E08081816021
:1043E0008083E8EDF0E080818F77808319BCA7EDB2
:1043F000B0E08C918E7F8C9380818F7E8083109231
:10440000D70208950F931F93CF93DF930E945622F4
:104410000E945E22C8EDD0E088818F7788838881F2
:104420008068888388818F7D888319BC1092D80228
:104430001092D4021092D6021092D50200EE10E033
:10444000F80180818B7F808388818160888342E04E
:1044500060E080E00E946121E1EEF0E080818E7FEB
:104460008083E2EEF0E080818160808380818860DB
:104470008083F80180818E7F80838881806188833A
:10448000DF91CF911F910F910895E8EDF0E08081C9
:104490008F7E8083E7EDF0E080818160808384E01F
:1044A00082BF81E08093D7020C940222E8EDF0E015
:1044B00080818E7F80831092E20008951092DA004E
:1044C0001092E10008951F920F920FB60F921124DF
:1044D0002F933F934F935F936F937F938F939F930C
:1044E000AF93BF93EF93FF938091E10082FF0BC0E6
:1044F0008091E20082FF07C08091E1008B7F809372
:10450000E1000E94D9248091DA0080FF1FC08091D1
:10451000D80080FF1BC08091DA008E7F8093DA0084
:104520008091D90080FF0DC080E189BD82E189BD05
:1045300009B400FEFDCF81E08093D8020E94A71E3F
:1045400005C019BC1092D8020E94B51E8091E100EE
:1045500080FF19C08091E20080FF15C08091E200C9
:104560008E7F8093E2008091E20080618093E20080
:104570008091D80080628093D80019BC85E0809338
:10458000D8020E94BA1E8091E10084FF30C0809161
:10459000E20084FF2CC080E189BD82E189BD09B4BD
:1045A00000FEFDCF8091D8008F7D8093D800809150
:1045B000E1008F7E8093E1008091E2008F7E809306
:1045C000E2008091E20081608093E2008091D40259
:1045D000882311F084E007C08091E30087FD02C0CA
:1045E00081E001C083E08093D8020E94C21E8091C6
:1045F000E10083FF29C08091E20083FF25C0809104
:10460000E100877F8093E10082E08093D8021092DE
:10461000D4028091E1008E7F8093E1008091E200DE
:104620008E7F8093E2008091E20080618093E200BF
:1046300042E060E080E00E9461218091F0008860AB
:104640008093F0000E94B81EFF91EF91BF91AF914F
:104650009F918F917F916F915F914F913F912F919A
:104660000F900FBE0F901F9018951F920F920FB6CC
:104670000F9211242F933F934F935F936F937F93E8
:104680008F939F93AF93BF93CF93DF93EF93FF935A
:10469000C091E900CF708091EC00D82FD17080FDDF
:1046A000D0E81092E9008091F000877F8093F000BD
:1046B00078940E9479231092E9008091F00088603C
:1046C0008093F000CD2BCF70C093E900FF91EF9164
:1046D000DF91CF91BF91AF919F918F917F916F911A
:1046E0005F914F913F912F910F900FBE0F901F90B0
:1046F00018951F93CF93DF93CDB7DEB7AA970FB668
:10470000F894DEBF0FBECDBFE9EDF2E08091F1007D
:10471000819322E0E13EF207C9F70E94E51E8091F5
:10472000E80083FF2EC18091D9029091DA02492FCF
:1047300050E04A30510508F024C1FA01E059FF4F1A
:104740000C941D25803821F0823809F01AC108C068
:104750008091D5029091D602992389F082600FC092
:104760008091DD028F70873008F00BC18093E900E3
:104770008091EB0085FB882780F91092E9009091E9
:10478000E800977F9093E8008093F1001092F10089
:10479000D1C0282F2D7F09F0F4C0882319F0823072
:1047A00061F0EFC08091DB02813009F0EAC0933004
:1047B00009F080E08093D6022EC08091DB02811147
:1047C0002AC08091DD028F702FEF280F263008F06D
:1047D000D8C08093E9002091EB0020FF1CC09330EB
:1047E00021F48091EB00806214C09091EB00906105
:1047F0009093EB0021E030E0A90102C0440F551F67
:104800008A95E2F74093EA001092EA008091EB006B
:1048100088608093EB001092E9008091E800877F28
:104820008093E8000E949621ACC08111AAC010912B
:10483000DB021F778091E3008078812B8093E30077
:104840008091E800877F8093E8000E949621809104
:10485000E80080FFFCCF8091E30080688093E30054
:10486000111102C082E001C083E08093D80289C0A8
:104870008058823008F085C08091DB029091DC0284
:104880008C3D53E0950779F583E08A838AE289833A
:104890004FB7F894DE01139620E03EE051E2E32F9B
:1048A000F0E050935700E49120FF03C0E295EF70D1
:1048B0003F5FEF708E2F90E0EA3010F0C79601C096
:1048C000C0968D939D932F5F243149F74FBF809100
:1048D000E800877F8093E8006AE270E0CE010196ED
:1048E0000E94A22016C06091DD027091DE02AE012E
:1048F0004F5F5F4F0E94E91FBC01892B09F441C043
:104900009091E800977F9093E80089819A810E94B6
:1049100000218091E8008B778093E80032C08038D6
:1049200081F58091E800877F8093E8008091D40230
:104930008093F1008091E8008E7772CF811121C0C1
:104940008091DB029091DC0299270297D4F4809148
:10495000E800877F8093E8008091DB028093D40297
:104960000E9496218091D402811106C08091E300BB
:1049700087FD02C081E001C084E08093D8020E94DC
:10498000CC1E8091E80083FF0AC08091E800877FF9
:104990008093E8008091EB0080628093EB00AA9600
:1049A0000FB6F894DEBF0FBECDBFDF91CF911F9140
:1049B00008950895CF938091D8028823A1F0C091E3
:1049C000E900CF709091EC00892F817090FD80E814
:1049D000C82B1092E9008091E80083FD0E947923A2
:1049E000CF70C093E900CF910895AA1BBB1B51E182
:1049F00007C0AA1FBB1FA617B70710F0A61BB70B4F
:104A0000881F991F5A95A9F780959095BC01CD01F3
:104A1000089597FB072E16F4009407D077FD09D070
:104A20000E94F52407FC05D03EF4909581959F4F98
:104A30000895709561957F4F0895EE0FFF1F0590C3
:104A4000F491E02D09940F931F93CF93DF9382305D
:104A5000910510F482E090E0E091E302F091E4022D
:104A600020E030E0A0E0B0E0309719F140815181C2
:104A70000281138148175907C8F08417950769F414
:104A8000109731F012960C93129713961C9327C02F
:104A90000093E3021093E40222C02115310519F0BE
:104AA0004217530718F49A01BD01EF01DF01F80125
:104AB000DBCF21153105F9F0281B390B24303105E6
:104AC00080F48A819B816115710521F0FB0193833C
:104AD000828304C09093E4028093E302FE01329645
:104AE00044C0FE01E20FF31F8193919322503109DC
:104AF000398328833AC02091E1023091E202232BCE
:104B000041F420910201309103013093E20220939D
:104B1000E10220910001309101012115310541F49C
:104B20002DB73EB74091040150910501241B350B70
:104B3000E091E102F091E202E217F307A0F42E1BEC
:104B40003F0B2817390778F0AC014E5F5F4F2417F1
:104B5000350748F04E0F5F1F5093E2024093E10289
:104B60008193919302C0E0E0F0E0CF01DF91CF911B
:104B70001F910F910895CF93DF93009709F481C09F
:104B8000FC01329713821282A091E302B091E402F9
:104B9000109781F420813181820F931F2091E102CF
:104BA0003091E2022817390751F5F093E202E093C1
:104BB000E10267C0ED0120E030E0CE17DF0740F4EE
:104BC0004A815B819E0141155105F1F0EA01F5CF63
:104BD000D383C28340815181840F951FC817D907A1
:104BE00059F488819981840F951F0296918380835F
:104BF0008A819B81938382832115310529F4F09367
:104C0000E402E093E3023DC0E901FB83EA834991BA
:104C10005991C40FD51FEC17FD0761F48081918174
:104C2000840F951F0296E90199838883828193817D
:104C30009B838A83E0E0F0E012968D919C9113971C
:104C4000009719F0FD01DC01F7CF8D919C91119730
:104C50009D012E5F3F4F820F931F2091E102309103
:104C6000E2022817390769F4309729F41092E40218
:104C70001092E30202C013821282B093E202A09368
:104C8000E102DF91CF910895FB01DC0104C08D9119
:104C90000190801921F441505040C8F7881B990BAE
:104CA0000895F999FECF92BD81BDF89A992780B5F4
:104CB0000895A6E1B0E044E050E00C948B26A8E112
:104CC000B0E042E050E00C948B26262FF999FECFFD
:104CD00092BD81BDF89A019700B4021639F01FBA4F
:104CE00020BD0FB6F894FA9AF99A0FBE089503966C
:104CF000272F0E9466260E946526252F0E94662681
:104D0000242F0C9466260196272F0E9466260C9469
:104D10006526DC01CB01FC01F999FECF06C0F2BD8E
:104D2000E1BDF89A319600B40D9241505040B8F769
:064D30000895F894FFCF86
:104D36000000E50220002000C80031023C071428CC
:104D46003C0714101E331E141EA31E9F1E131E01A5
:104D5600E200E900EA00B500B600B700CD00830125
:104D6600CC008A0192019401210223022402250229
:104D7600260227022A02B300B4006F007000818267
:104D860083E200E900EA00B500B600B700CD008373
:104D960001CC008A019201940121022302240225FA
:104DA60002260227022A02B300B4006F00700081B7
:104DB600828340476D2405DD0470041C0435044ECF
:024DC6000400E7
:00000001FF
